:020000040000FA
:0408000070EF09F09C
:1008100003B284EF05F0F2B4A2EF05F09EB0AAEFA8
:1008200005F09EB2B2EF05F0F2A81AEF04F0F2B2B2
:1008300032EF04F09EB61FEF04F01FEF09F09E9612
:1008400000011450000A06E000011450010A06E0FD
:100850001FEF09F01CEC21F01FEF09F014EC23F05E
:100860001FEF09F0CD90F2929EA03CEF04F0010141
:10087000533F3CEF04F0542BB2C1B6F1B3C1B7F112
:10088000B4C1B8F1B5C1B9F1AEC1B2F1AFC1B3F104
:10089000B0C1B4F1B1C1B5F1AAC1AEF1ABC1AFF114
:1008A000ACC1B0F1ADC1B1F1A6C1AAF1A7C1ABF124
:1008B000A8C1ACF1A9C1ADF1A2C1A6F1A3C1A7F134
:1008C000A4C1A8F1A5C1A9F19EC1A2F19FC1A3F144
:1008D000A0C1A4F1A1C1A5F19AC19EF19BC19FF154
:1008E0009CC1A0F19DC1A1F1CECF9AF1CFCF9BF1D8
:1008F00053C19CF154C19DF1CF6ACE6A0101536B83
:10090000546B9E90CD800FBC0F8E0FBA8BEF04F00E
:100910000F8A1FEF09F013880F8C0FBEC8EF04F089
:100920009AC19EF19BC19FF19CC1A0F19DC1A1F113
:100930009EC1A2F19FC1A3F1A0C1A4F1A1C1A5F1E3
:10094000A2C1A6F1A3C1A7F1A4C1A8F1A5C1A9F1B3
:10095000A6C1AAF1A7C1ABF1A8C1ACF1A9C1ADF183
:10096000AAC1AEF1ABC1AFF1ACC1B0F1ADC1B1F153
:10097000AEC1B2F1AFC1B3F1B0C1B4F1B1C1B5F123
:10098000B2C1B6F1B3C1B7F1B4C1B8F1B5C1B9F1F3
:1009900001015E6B5F6B606B616B9A515E279B51CF
:1009A0005F239C5160239D5161239E515E279F517F
:1009B0005F23A0516023A1516123A2515E27A3515F
:1009C0005F23A4516023A5516123A6515E27A7513F
:1009D0005F23A8516023A9516123AA515E27AB511F
:1009E0005F23AC516023AD516123AE515E27AF51FF
:1009F0005F23B0516023B1516123B2515E27B351DF
:100A00005F23B4516023B5516123B6515E27B751BE
:100A10005F23B8516023B9516123D890010161333C
:100A200060335F335E33D8900101613360335F33ED
:100A30005E33D8900101613360335F335E3300C1B0
:100A40000CF101C10DF102C10EF103C10FF104C19E
:100A500010F105C111F106C112F107C113F108C16E
:100A600014F109C115F10AC116F10BC117F134C116
:100A700035F111B847EF05F00101620E046F010E68
:100A8000056F000E066F000E076F50EF05F00101B5
:100A9000A70E046F020E056F000E066F000E076FA3
:100AA0005EC100F15FC101F160C102F161C103F1FA
:100AB000B3EC1FF003BF04D019BE02D019A0108CF4
:100AC00011A068EF05F010BA68EF05F00F80108AEA
:100AD0000CC100F10DC101F10EC102F10FC103F112
:100AE00010C104F111C105F112C106F113C107F1E2
:100AF00014C108F115C109F116C10AF117C10BF1B2
:100B000035C134F11FEF09F00392ABB2AB98AB885B
:100B1000030103EE00F080517F0BE92604C0EFFFD4
:100B2000802B8151805D700BD8A48B820000805196
:100B3000815D700BD8A48B9281518019D8B4079035
:100B40001FEF09F0F2940101453F1FEF09F0462B1A
:100B50001FEF09F09E900101533F1FEF09F0542B46
:100B60001FEF09F09E9211B827EF07F08BB4C0EF8A
:100B700005F010ACC0EF05F08B84109CC1EF05F0C0
:100B80008B94C3CF55F1C4CF56F1C28207B430EF76
:100B900006F047C14BF148C14CF149C14DF14AC182
:100BA0004EF15EC162F15FC163F160C164F161C188
:100BB00065F113A8DEEF05F0138C13989AC1BAF112
:100BC0009BC1BBF19CC1BCF19DC1BDF19EC1BEF1F9
:100BD0009FC1BFF1A0C1C0F1A1C1C1F1A2C1C2F1C9
:100BE000A3C1C3F1A4C1C4F1A5C1C5F1A6C1C6F199
:100BF000A7C1C7F1A8C1C8F1A9C1C9F1AAC1CAF169
:100C0000ABC1CBF1ACC1CCF1ADC1CDF1AEC1CEF138
:100C1000AFC1CFF1B0C1D0F1B1C1D1F1B2C1D2F108
:100C2000B3C1D3F1B4C1D4F1B5C1D5F1B6C1D6F1D8
:100C3000B7C1D7F1B8C1D8F1B9C1D9F10101555146
:100C40005B2756515C23E86A5D230E2E30EF06F0D9
:100C50005CC157F15DC158F15B6B5C6B5D6B078EDE
:100C60000201002F1FEF09F03C0E006F1A50E00B3D
:100C7000E00AE866128818BE02D018B4108E00C1CF
:100C80000CF101C10DF102C10EF103C10FF104C15C
:100C900010F105C111F106C112F107C113F108C12C
:100CA00014F109C115F10AC116F10BC117F134C1D4
:100CB00035F101018E6764EF06F08F6764EF06F08F
:100CC000906764EF06F0916768EF06F098EF06F022
:100CD00092C100F193C101F194C102F195C103F1F8
:100CE0000101010E046F000E056F000E066F000E6D
:100CF000076FB3EC1FF000C192F101C193F102C183
:100D000094F103C195F100678DEF06F001678DEF57
:100D100006F002678DEF06F0036798EF06F08EC1CC
:100D200092F18FC193F190C194F191C195F10F802F
:100D3000D57ED5BE6ED0D6CF47F1D7CF48F145C1CD
:100D400049F1E86AE8CF4AF1138A19BE02D019A026
:100D5000108C109047C100F148C101F149C102F166
:100D60004AC103F101010A0E046F000E056F000E67
:100D7000066F000E076FB3EC1FF003AF1080010188
:100D800054A7CFEF06F00F9A0F9C0F9E0101000EA3
:100D90005E6F600E5F6F3D0E606F080E616F010148
:100DA00047BFDFEF06F04867DFEF06F04967DFEF88
:100DB00006F04A67DFEF06F0F28804EF07F0F298DA
:100DC0005E6B5F6B606B616B9A6B9B6B9C6B9D6BDF
:100DD0009E6B9F6BA06BA16BA26BA36BA46BA56BAF
:100DE000A66BA76BA86BA96BAA6BAB6BAC6BAD6B5F
:100DF000AE6BAF6BB06BB16BB26BB36BB46BB56B0F
:100E0000B66BB76BB86BB96BD76AD66A0101456B25
:100E1000466B0CC100F10DC101F10EC102F10FC111
:100E200003F110C104F111C105F112C106F113C1A2
:100E300007F114C108F115C109F116C10AF117C172
:100E40000BF135C134F11FEF09F01FEF09F002017A
:100E5000002F81EF08F0D59ED6CF47F1D7CF48F1CC
:100E600045C149F1E86AE8CF4AF1138AD76AD66AE0
:100E70000101456B466BD58E1A50E00BE00AE8661F
:100E8000128818BE02D018B4108E17AE1C8C00C188
:100E90000CF101C10DF102C10EF103C10FF104C14A
:100EA00010F105C111F106C112F107C113F108C11A
:100EB00014F109C115F10AC116F10BC117F134C1C2
:100EC00035F10FA0109A11B871EF07F00101620E11
:100ED000046F010E056F000E066F000E076F7AEFAC
:100EE00007F00101A70E046F020E056F000E066FDA
:100EF000000E076F47C100F148C101F149C102F17D
:100F00004AC103F1B3EC1FF003BF8DEF07F019BE28
:100F100002D019A0108C11B00F800CC100F10DC1CE
:100F200001F10EC102F10FC103F110C104F111C1B1
:100F300005F112C106F113C107F114C108F115C181
:100F400009F116C10AF117C10BF135C134F10201E3
:100F50003C0E006F00C10CF101C10DF102C10EF198
:100F600003C10FF104C110F105C111F106C112F165
:100F700007C113F108C114F109C115F10AC116F135
:100F80000BC117F134C135F101018E67CFEF07F0C6
:100F90008F67CFEF07F09067CFEF07F09167D3EF40
:100FA00007F003EF08F092C100F193C101F194C181
:100FB00002F195C103F10101010E046F000E056FEE
:100FC000000E066F000E076FB3EC1FF000C192F128
:100FD00001C193F102C194F103C195F10067F8EFEB
:100FE00007F00167F8EF07F00267F8EF07F0036713
:100FF00003EF08F08EC192F18FC193F190C194F18B
:1010000091C195F10F80109047C100F148C101F1E5
:1010100049C102F14AC103F101010A0E046F000E39
:10102000056F000E066F000E076FB3EC1FF003AFE5
:101030001080010154A729EF08F00F9A0F9C0F9E12
:101040000101000E5E6F600E5F6F3D0E606F080E57
:10105000616F47C100F148C101F149C102F14AC1C4
:1010600003F10101140E046F050E056F000E066FEB
:10107000000E076FB3EC1FF003AF42EF08F0F288E9
:1010800067EF08F0F2985E6B5F6B606B616B9A6B59
:101090009B6B9C6B9D6B9E6B9F6BA06BA16BA26B04
:1010A000A36BA46BA56BA66BA76BA86BA96BAA6BB4
:1010B000AB6BAC6BAD6BAE6BAF6BB06BB16BB26B64
:1010C000B36BB46BB56BB66BB76BB86BB96B0CC16C
:1010D00000F10DC101F10EC102F10FC103F110C108
:1010E00004F111C105F112C106F113C107F114C1D8
:1010F00008F115C109F116C10AF117C10BF135C18B
:1011000034F1D3EC23F01D661ED01CAE11D01C9E12
:101110001D8E18AE07D0146A040E156E166A1CECEC
:1011200021F011D0146A156A166A1CEC21F00BD05C
:101130001CAC09D01C9C1D8C010E146E156A166A1D
:1011400014EC23F000D08BB4ADEF08F010ACADEF91
:1011500008F08B84109CAEEF08F08B94C3CF55F150
:10116000C4CF56F1C28207B41DEF09F047C14BF15D
:1011700048C14CF149C14DF14AC14EF15EC162F125
:101180005FC163F160C164F161C165F113A8CBEF88
:1011900008F0138C13989AC1BAF19BC1BBF19CC1A2
:1011A000BCF19DC1BDF19EC1BEF19FC1BFF1A0C107
:1011B000C0F1A1C1C1F1A2C1C2F1A3C1C3F1A4C1D7
:1011C000C4F1A5C1C5F1A6C1C6F1A7C1C7F1A8C1A7
:1011D000C8F1A9C1C9F1AAC1CAF1ABC1CBF1ACC177
:1011E000CCF1ADC1CDF1AEC1CEF1AFC1CFF1B0C147
:1011F000D0F1B1C1D1F1B2C1D2F1B3C1D3F1B4C117
:10120000D4F1B5C1D5F1B6C1D6F1B7C1D7F1B8C1E6
:10121000D8F1B9C1D9F1010155515B2756515C2371
:10122000E86A5D230E2E1DEF09F05CC157F15DC128
:1012300058F15B6B5C6B5D6B078E1FEF09F002C0B2
:10124000E0FF005001C0D8FF1000A6B225EF09F062
:101250000CC0A9FF0BC0A8FFA69EA69CA684F29E68
:10126000550EA76EAA0EA76EA682F28EA694A6B2FF
:1012700037EF09F00C2A1200A96EA69EA69CA68044
:10128000A8500C2A120004012C0E826F48EC0BF0BF
:10129000AEEC20F00C503CEC09F0E8CF00F10C5023
:1012A0003CEC09F0E8CF01F101AF5CEF09F001017E
:1012B000FF0E026FFF0E036F51EC20F0296768EFFD
:1012C00009F00401200E826F48EC0BF06DEF09F07D
:1012D00004012D0E826F48EC0BF05BEC1EF0120047
:1012E000306A076A0F6A106A116A126A136A0F017C
:1012F0000E0EC16E860EC06E030EC26E0F01896A9D
:10130000110E926E080E8A6EF10E936E8B6A980E15
:10131000946EF18EFC0E3CEC09F0E8CF0BF00BA0C4
:1013200011800BA211820BA411840BA81188C90E85
:101330003CEC09F0E8CF17F0CA0E3CEC09F0E8CF1E
:1013400018F0CB0E3CEC09F0E8CF19F0CC0E3CECD9
:1013500009F0E8CF1AF0CD0E3CEC09F0E8CF2FF001
:101360001C6A1D6A0E6A01015B6B5C6B5D6B576BDF
:10137000586BF29A0101476B486B496B4A6B4B6B98
:101380004C6B4D6B4E6B4F6B506B516B526B456B97
:10139000466BD76AD66A0F01280ED56EF28A9D90E9
:1013A000B00ECD6E01015E6B5F6B606B616B626B4B
:1013B000636B646B656B666B676B686B696B536BB8
:1013C000546BCF6ACE6A0F9A0F9C0F9E9D80760E4B
:1013D000CA6E9D8202013C0E006FCC6A160E3CEC78
:1013E00009F0E8CF00F1170E3CEC09F0E8CF01F16D
:1013F000180E3CEC09F0E8CF02F1190E3CEC09F0B4
:10140000E8CF03F1010103AF20EF0AF0AEEC20F0CA
:10141000160E0C6E00C10BF025EC09F0170E0C6EC9
:1014200001C10BF025EC09F0180E0C6E02C10BF097
:1014300025EC09F0190E0C6E03C10BF025EC09F038
:1014400000C18EF101C18FF102C190F103C191F190
:1014500000C192F101C193F102C194F103C195F170
:101460001A0E3CEC09F0E8CF00F11B0E3CEC09F041
:10147000E8CF01F11C0E3CEC09F0E8CF02F11D0EA3
:101480003CEC09F0E8CF03F1010103AF76EF0AF07D
:10149000AEEC20F01A0E0C6E00C10BF025EC09F03A
:1014A0001B0E0C6E01C10BF025EC09F01C0E0C6E2E
:1014B00002C10BF025EC09F01D0E0C6E03C10BF000
:1014C00025EC09F01A0E3CEC09F0E8CF00F11B0EF8
:1014D0003CEC09F0E8CF01F11C0E3CEC09F0E8CF40
:1014E00002F11D0E3CEC09F0E8CF03F100C196F1CA
:1014F00001C197F102C198F103C199F1240EAC6EBC
:10150000900EAB6E240EAC6E080EB86E000EB06E70
:101510001F0EAF6E0401806B816B0F01900EAB6EDE
:101520000F019D8A0301806B816BC26B8B92146AE1
:10153000156A166A9D8607900001F28EF28C07B03C
:1015400004EF1DF00FB017EF16F010BE17EF16F0F6
:1015500012B817EF16F00301805181197F0BD8B430
:1015600004EF1DF013EE00F081517F0BE126812B7B
:10157000E7CFE8FFE00BD8B404EF1DF023EE82F0D4
:10158000C2513F0BD926E7CFDFFFC22BDF50780ACD
:10159000D8A404EF1DF0078092C100F193C101F1BE
:1015A00094C102F195C103F10101040E046F000E14
:1015B000056F000E066F000E076FB3EC1FF000AF53
:1015C000EBEF0AF00101030E926F000E936F000E15
:1015D000946F000E956F03018251720AD8B4F3EF35
:1015E00015F08251520AD8B4F3EF15F08251750A02
:1015F000D8B4F3EF15F08251630AD8B4BEEF19F0F6
:101600008251690AD8B495EF12F082517A0AD8B49F
:10161000A8EF13F08251490AD8B434EF12F0825186
:10162000500AD8B43EEF11F08251700AD8B486EF58
:1016300011F08251540AD8B4B6EF11F08251740AF5
:10164000D8B401EF12F08251410AD8B45EEF0CF029
:1016500082514B0AD8B45CEF0BF082516D0AD8B4BA
:1016600091EF10F082514D0AD8B4AAEF10F08251D8
:10167000730AD8B423EF15F08251530AD8B488EF17
:1016800015F08251590AD8B4E2EF0FF0F5EF19F0D6
:10169000040114EE00F080517F0BE12682C4E7FFC5
:1016A000802B120004010D0E826F48EC0BF00A0E25
:1016B000826F48EC0BF0120004014B0E826F48EC75
:1016C0000BF004012C0E826F48EC0BF081B802D0B5
:1016D0002FB630D003018351430AD8B4A1EF0BF0E9
:1016E00003018351630AD8B4A3EF0BF003018351C4
:1016F000520AD8B4A5EF0BF003018351720AD8B493
:10170000A7EF0BF003018351470AD8B4A9EF0BF000
:1017100003018351670AD8B4ABEF0BF00301835187
:10172000540AD8B4ADEF0BF003018351740AD8B456
:101730001CEF0CF003018351550AD8B4AFEF0BF046
:1017400082D02F807AD02F9078D02F8276D02F928F
:1017500074D02F8472D02F9470D02F866ED084C313
:1017600030F185C331F186C332F187C333F1010112
:10177000296BFCEC20F073EC20F000C104F101C1F6
:1017800005F102C106F103C107F1EFEC20F0200ED4
:10179000F86EF76AF66A0900F5CF2CF10900F5CF6B
:1017A0002DF10900F5CF2EF10900F5CF2FF1090039
:1017B000F5CF30F10900F5CF31F10900F5CF32F165
:1017C0000900F5CF33F10101296BFCEC20F073EC3B
:1017D00020F0B3EC1FF00067F5EF0BF00167F5EFB9
:1017E0000BF00267F5EF0BF0036701D025D0040181
:1017F0004E0E826F48EC0BF004016F0E826F48ECC6
:101800000BF004014D0E826F48EC0BF00401610EE9
:10181000826F48EC0BF00401740E826F48EC0BF001
:101820000401630E826F48EC0BF00401680E826FB6
:1018300048EC0BF0F3EF19F02F96CD0E0C6E2FC085
:101840000BF025EC09F0CD0E3CEC09F0E8CF2FF0C1
:101850002FB006D00401630E826F48EC0BF005D068
:101860000401430E826F48EC0BF02FB206D0040146
:10187000720E826F48EC0BF005D00401520E826F9D
:1018800048EC0BF02FB406D00401670E826F48ECD1
:101890000BF005D00401470E826F48EC0BF02FB619
:1018A00006D00401740E826F48EC0BF005D00401E1
:1018B000540E826F48EC0BF0F3EF19F00401410E67
:1018C000826F48EC0BF003018351310AD8B402EF68
:1018D0000FF003018351320AD8B432EF0EF0030146
:1018E0008351330AD8B4BBEF0DF003018351340A9E
:1018F000D8B4ABEF0CF003018351350AD8B488EFAC
:101900000CF004013F0E826F48EC0BF0F3EF19F07E
:1019100004012C0E826F48EC0BF003018451300A55
:10192000D8B49BEF0CF003018451310AD8B4A3EF73
:101930000CF0F4EF0DF08B900401300E826F48EC48
:101940000BF0A9EF0CF08B800401310E826F48EC94
:101950000BF0F3EF19F0CC0E3CEC09F0E8CF0BF0F4
:1019600004012C0E826F48EC0BF003018451310A04
:10197000D8B4CFEF0CF003018451300AD8B4D1EFC2
:101980000CF0030184514D0AD8B4DBEF0CF00301D5
:101990008451540AD8B4E2EF0CF0F9EF0CF08A84C9
:1019A00001D08A940BAE04D00BAC02D00BBA21D07C
:1019B000E00E0B1218D01F0E0B168539E844E00B11
:1019C0000B1211D0E00E0B16EFEC20F085C332F1B4
:1019D00086C333F10101296BFCEC20F073EC20F09D
:1019E00000511F0B0B12CC0E0C6E0BC00BF025EC34
:1019F00009F00401340E826F48EC0BF004012C0E48
:101A0000826F48EC0BF0CC0E3CEC09F0E8CF1AF0FA
:101A10008AB406D00401300E826F48EC0BF005D07A
:101A20000401310E826F48EC0BF004012C0E826F22
:101A300048EC0BF01A38E840070BE8CF82F40401B9
:101A4000300E822748EC0BF004012C0E826F48EC1C
:101A50000BF0AEEC20F01A501F0BE8CF00F151EC68
:101A600020F032C182F40401300E822748EC0BF0E2
:101A700033C182F40401300E822748EC0BF00401DC
:101A80002C0E826F48EC0BF0AEEC20F02DC000F174
:101A900000AF0BD0FF0E016FFF0E026FFF0E036F42
:101AA00004012D0E826F48EC0BF051EC20F031C197
:101AB00082F40401300E822748EC0BF032C182F42C
:101AC0000401300E822748EC0BF033C182F404018C
:101AD000300E822748EC0BF004012C0E826F48EC8C
:101AE0000BF0AEEC20F02CC000F151EC20F031C135
:101AF00082F40401300E822748EC0BF032C182F4EC
:101B00000401300E822748EC0BF033C182F404014B
:101B1000300E822748EC0BF004012C0E826F48EC4B
:101B20000BF0AEEC20F02EC000F100AF0BD0FF0E9A
:101B3000016FFF0E026FFF0E036F04012D0E826F07
:101B400048EC0BF051EC20F031C182F40401300E6E
:101B5000822748EC0BF032C182F40401300E822758
:101B600048EC0BF033C182F40401300E822748ECBC
:101B70000BF0F3EF19F0CB0E3CEC09F0E8CF0BF0D3
:101B800004012C0E826F48EC0BF003018451450ACE
:101B9000D8B4DFEF0DF003018451440AD8B4E2EF6A
:101BA0000DF003018451300AD8B4E5EF0DF00301C4
:101BB0008451310AD8B4E9EF0DF0F4EF0DF00B9E2B
:101BC000EEEF0DF00B8EEEEF0DF0FC0E0B16EEEFC0
:101BD0000DF0FC0E0B160B80EEEF0DF0CB0E0C6E25
:101BE0000BC00BF025EC09F00401330E826F48ECBA
:101BF0000BF004012C0E826F48EC0BF0CB0E3CEC8A
:101C000009F0E8CF19F019BE0DEF0EF00401450EF2
:101C1000826F48EC0BF012EF0EF00401440E826F5D
:101C200048EC0BF004012C0E826F48EC0BF0040121
:101C3000300E826F48EC0BF004012C0E826F48ECE2
:101C40000BF019B02BEF0EF00401300E826F48EC50
:101C50000BF030EF0EF00401310E826F48EC0BF008
:101C6000F3EF19F0CA0E3CEC09F0E8CF0BF00401D9
:101C70002C0E826F48EC0BF003018451450AD8B456
:101C80006EEF0EF003018451440AD8B471EF0EF0E8
:101C9000030184514D0AD8B47AEF0EF00301845148
:101CA000410AD8B474EF0EF003018451460AD8B447
:101CB00077EF0EF003018451560AD8B482EF0EF08C
:101CC00003018451500AD8B48DEF0EF00301845102
:101CD000520AD8B490EF0EF099EF0EF00B9E93EFEE
:101CE0000EF00B8E93EF0EF00B9C93EF0EF00B8C1F
:101CF00093EF0EF0FC0E0B1685C3E8FF030B0B12DF
:101D000093EF0EF0C70E0B1685C3E8FF070BE846EE
:101D1000E846E8460B1293EF0EF00B8493EF0EF0BB
:101D20000B9493EF0EF0CA0E0C6E0BC00BF025EC6B
:101D300009F0CA0E3CEC09F0E8CF18F00401320EAD
:101D4000826F48EC0BF004012C0E826F48EC0BF014
:101D500018BEB2EF0EF00401450E826F48EC0BF096
:101D6000B7EF0EF00401440E826F48EC0BF0040153
:101D70002C0E826F48EC0BF018C0E8FF030BE8CF85
:101D800082F40401300E822748EC0BF004012C0E83
:101D9000826F48EC0BF018BCD5EF0EF00401410E39
:101DA000826F48EC0BF0DAEF0EF00401460E826F02
:101DB00048EC0BF004012C0E826F48EC0BF018C0BD
:101DC000E8FF380BE842E842E842E8CF82F4040139
:101DD000300E822748EC0BF004012C0E826F48EC89
:101DE0000BF018B4FBEF0EF00401520E826F48ECBA
:101DF0000BF000EF0FF00401500E826F48EC0BF077
:101E0000F3EF19F0C90E3CEC09F0E8CF0BF0040138
:101E10002C0E826F48EC0BF003018451450AD8B4B4
:101E200020EF0FF003018451440AD8B423EF0FF0E0
:101E3000030184514D0AD8B426EF0FF034EF0FF0B0
:101E40000B9E2EEF0FF00B8E2EEF0FF0F80E0B16F1
:101E500085C3E8FF070B0B122EEF0FF0C90E0C6EB7
:101E60000BC00BF025EC09F00401310E826F48EC39
:101E70000BF004012C0E826F48EC0BF0C90E3CEC09
:101E800009F0E8CF17F017BE06D00401450E826FA7
:101E900048EC0BF005D00401440E826F48EC0BF0C7
:101EA00004012C0E826F48EC0BF017C0E8FF070B03
:101EB000E8CF82F40401300E822748EC0BF00401D5
:101EC0002C0E826F48EC0BF00780AEEC20F028C09F
:101ED000E8FF003B00430043030B51EC20F033C10B
:101EE00082F40401300E822748EC0BF004012C0E22
:101EF000826F48EC0BF0AEEC20F028C001F1019F9E
:101F0000019D29C000F1010151EC20F02FC182F4A4
:101F10000401300E822748EC0BF030C182F404013A
:101F2000300E822748EC0BF031C182F40401300EF0
:101F3000822748EC0BF032C182F40401300E822774
:101F400048EC0BF033C182F40401300E822748ECD8
:101F50000BF004012C0E826F48EC0BF0AEEC20F07D
:101F60002AC001F12BC000F1D89001330033D89082
:101F700001330033010151EC20F02FC182F4040140
:101F8000300E822748EC0BF030C182F40401300E91
:101F9000822748EC0BF031C182F40401300E822715
:101FA00048EC0BF032C182F40401300E822748EC79
:101FB0000BF033C182F40401300E822748EC0BF0A1
:101FC000F3EF19F0FC0E3CEC09F0E8CF0BF0030145
:101FD0008351520AD8B419EF10F003018351720AE9
:101FE000D8B41CEF10F003018351500AD8B41FEF8E
:101FF00010F003018351700AD8B422EF10F00301EE
:102000008351550AD8B425EF10F003018351750AA6
:10201000D8B428EF10F003018351430AD8B431EF4C
:1020200010F003018351630AD8B434EF10F03DEF90
:1020300010F00B9037EF10F00B8037EF10F00B9291
:1020400037EF10F00B8237EF10F00B9437EF10F0F2
:102050000B8437EF10F00B9637EF10F00B8637EF4D
:1020600010F00B9837EF10F00B8837EF10F0FC0EE4
:102070000C6E0BC00BF025EC09F00401590E826FB9
:1020800048EC0BF01190119211941198FC0E3CEC5D
:1020900009F0E8CF0BF00BA011800BA211820BA46A
:1020A00011840BA8118811A05DEF10F00401520EED
:1020B000826F48EC0BF062EF10F00401720E826F39
:1020C00048EC0BF011A86CEF10F00401430E826F86
:1020D00048EC0BF071EF10F00401630E826F48ECD6
:1020E0000BF011A27BEF10F00401500E826F48EC50
:1020F0000BF080EF10F00401700E826F48EC0BF0D3
:1021000011A48AEF10F00401550E826F48EC0BF019
:102110008FEF10F00401750E826F48EC0BF0F3EFB7
:1021200019F004016D0E826F48EC0BF0030183512E
:10213000300AD8B4EEEF10F003018351310AD8B45D
:1021400001EF11F003018351320AD8B414EF11F0FA
:10215000F5EF19F081B803D02FB4F3EF19F00401B3
:102160004D0E826F48EC0BF0EFEC20F084C331F1A0
:1021700085C332F186C333F10101296BFCEC20F0F9
:1021800073EC20F003018351300AD8B4D6EF10F07D
:1021900003018351310AD8B4DEEF10F003018351FB
:1021A000320AD8B4E6EF10F0F5EF19F0FD0E0C6E20
:1021B00000C10BF025EC09F0EEEF10F0FE0E0C6EF6
:1021C00000C10BF025EC09F001EF11F0FF0E0C6ED1
:1021D00000C10BF025EC09F014EF11F00401300EF2
:1021E000826F48EC0BF004012C0E826F48EC0BF070
:1021F000AEEC20F0FD0E3CEC09F0E8CF00F125EF4D
:1022000011F00401310E826F48EC0BF004012C0E2A
:10221000826F48EC0BF0AEEC20F0FE0E3CEC09F0C7
:10222000E8CF00F125EF11F00401320E826F48EC87
:102230000BF0AEEC20F004012C0E826F48EC0BF09A
:10224000FF0E3CEC09F0E8CF00F151EC20F031C179
:1022500082F40401300E822748EC0BF032C182F484
:102260000401300E822748EC0BF033C182F40401E4
:10227000300E822748EC0BF0F3EF19F081B803D051
:102280002FB234EF12F083C32AF184C32BF185C33C
:102290002CF186C32DF187C32EF188C32FF189C39A
:1022A00030F18AC331F18BC332F18CC333F10101B8
:1022B000FCEC20F073EC20F0160E0C6E00C10BF05D
:1022C00025EC09F0170E0C6E01C10BF025EC09F09E
:1022D000180E0C6E02C10BF025EC09F0190E0C6EF5
:1022E00003C10BF025EC09F000C18EF101C18FF1A3
:1022F00002C190F103C191F100C192F101C193F1CA
:1023000002C194F103C195F134EF12F081B803D00A
:102310002FB234EF12F083C32AF184C32BF185C3AB
:102320002CF186C32DF187C32EF188C32FF189C309
:1023300030F18AC331F18BC332F18CC333F1010127
:10234000FCEC20F073EC20F000C18EF101C18FF1A4
:1023500002C190F103C191F100C192F101C193F169
:1023600002C194F103C195F134EF12F081B803D0AA
:102370002FB234EF12F083C32AF184C32BF185C34B
:102380002CF186C32DF187C32EF188C32FF189C3A9
:1023900030F18AC331F18CC332F18DC333F10101C5
:1023A000FCEC20F073EC20F00101000E046F000E35
:1023B000056F010E066F000E076FC4EC1FF01A0EBA
:1023C0000C6E00C10BF025EC09F01B0E0C6E01C168
:1023D0000BF025EC09F01C0E0C6E02C10BF025EC85
:1023E00009F01D0E0C6E03C10BF025EC09F000C1C5
:1023F00096F101C197F102C198F103C199F134EF4F
:1024000012F081B803D02FB234EF12F083C32AF157
:1024100084C32BF185C32CF186C32DF187C32EF124
:1024200088C32FF189C330F18AC331F18CC332F1F3
:102430008DC333F10101FCEC20F073EC20F00101BD
:10244000000E046F000E056F010E066F000E076F81
:10245000C4EC1FF000C196F101C197F102C198F1DF
:1024600003C199F134EF12F0160E3CEC09F0E8CFFD
:1024700000F1170E3CEC09F0E8CF01F1180E3CEC2E
:1024800009F0E8CF02F1190E3CEC09F0E8CF03F1B6
:1024900051EC20F014EC1EF00401730E826F48EC36
:1024A0000BF004012C0E826F48EC0BF08EC100F192
:1024B0008FC101F190C102F191C103F151EC20F003
:1024C00014EC1EF00401730E826F48EC0BF0040153
:1024D0002C0E826F48EC0BF01A0E3CEC09F0E8CFA2
:1024E00000F11B0E3CEC09F0E8CF01F11C0E3CECB6
:1024F00009F0E8CF02F11D0E3CEC09F0E8CF03F142
:1025000010EC1AF004012C0E826F48EC0BF096C10F
:1025100000F197C101F198C102F199C103F110ECEA
:102520001AF052EC0BF0F5EF19F00401690E826F0E
:1025300048EC0BF004012C0E826F48EC0BF001010B
:10254000040E006F000E016F000E026F000E036F8D
:1025500051EC20F02CC182F40401300E822748ECAB
:102560000BF02DC182F40401300E822748EC0BF0F1
:102570002EC182F40401300E822748EC0BF02FC1EB
:1025800082F40401300E822748EC0BF030C182F453
:102590000401300E822748EC0BF031C182F40401B3
:1025A000300E822748EC0BF032C182F40401300E69
:1025B000822748EC0BF033C182F40401300E8227ED
:1025C00048EC0BF004012C0E826F48EC0BF001017B
:1025D000030E006F000E016F000E026F000E036FFE
:1025E00051EC20F02CC182F40401300E822748EC1B
:1025F0000BF02DC182F40401300E822748EC0BF061
:102600002EC182F40401300E822748EC0BF02FC15A
:1026100082F40401300E822748EC0BF030C182F4C2
:102620000401300E822748EC0BF031C182F4040122
:10263000300E822748EC0BF032C182F40401300ED8
:10264000822748EC0BF033C182F40401300E82275C
:1026500048EC0BF004012C0E826F48EC0BF00101EA
:102660003A0E006F000E016F000E026F000E036F36
:1026700051EC20F02CC182F40401300E822748EC8A
:102680000BF02DC182F40401300E822748EC0BF0D0
:102690002EC182F40401300E822748EC0BF02FC1CA
:1026A00082F40401300E822748EC0BF030C182F432
:1026B0000401300E822748EC0BF031C182F4040192
:1026C000300E822748EC0BF032C182F40401300E48
:1026D000822748EC0BF033C182F40401300E8227CC
:1026E00048EC0BF004012C0E826F48EC0BF0200E2E
:1026F000F86EF76AF66A04010900F5CF82F448EC37
:102700000BF00900F5CF82F448EC0BF00900F5CF8F
:1027100082F448EC0BF00900F5CF82F448EC0BF0A2
:102720000900F5CF82F448EC0BF00900F5CF82F4F4
:1027300048EC0BF00900F5CF82F448EC0BF00900EF
:10274000F5CF82F448EC0BF052EC0BF0F5EF19F0FA
:1027500081B803D02FB0F8EF13F08351630AD8A4E7
:10276000F3EF19F08451610AD8A4F3EF19F0855101
:102770006C0AD8A4F3EF19F08651410A42E0865161
:10278000440A1BE08651420AD8B414EF14F0865173
:10279000350AD8B47FEF1BF08651360AD8B4D4EF8F
:1027A0001BF08651370AD8B43DEF1CF08651380A29
:1027B000D8B49BEF1CF0F3EF19F00798079A0401C7
:1027C0007A0E826F48EC0BF00401780E826F48ECB1
:1027D0000BF00401640E826F48EC0BF081A8F8EF57
:1027E00013F00401550E826F48EC0BF0FDEF13F06F
:1027F00004014C0E826F48EC0BF052EC0BF0F5EF3D
:1028000019F00788079A04017A0E826F48EC0BF0E2
:102810000401410E826F48EC0BF00401610E826FDF
:1028200048EC0BF0EEEF13F00798078A04017A0EDC
:10283000826F48EC0BF00401420E826F48EC0BF003
:102840000401610E826F48EC0BF0EEEF13F0010112
:10285000666732EF14F0676732EF14F0686732EFA3
:1028600014F0696715D04F673DEF14F050673DEFE6
:1028700014F051673DEF14F052670AD00101000EC9
:10288000006F000E016F000E026F000E036F12004A
:1028900011B80AD00101620E046F010E056F000E1F
:1028A000066F000E076F09D00101A70E046F020E1C
:1028B000056F000E066F000E076F66C100F167C15D
:1028C00001F168C102F169C103F1B3EC1FF003BF6C
:1028D000DAEF14F0119A119C0101000E046FA80E9A
:1028E000056F550E066F020E076F66C100F167C1D6
:1028F00001F168C102F169C103F166C18AF167C1E2
:102900008BF168C18CF169C18DF1B3EC1FF003BF8D
:102910000BD00101000E8A6FA80E8B6F550E8C6FC5
:10292000020E8D6F118A119C0E0E3CEC09F0E8CF5F
:1029300018F10F0E3CEC09F0E8CF19F1100E3CEC49
:1029400009F0E8CF1AF1110E3CEC09F0E8CF1BF1C9
:10295000FCEC1EF08AC104F18BC105F18CC106F1BB
:102960008DC107F1B3EC1FF00782C0EC1EF0FCEC48
:102970001EF00792C0EC1EF08AC100F18BC101F17C
:102980008CC102F18DC103F10792C0EC1EF0CC0E98
:10299000046FE00E056F870E066F050E076FB3EC30
:1029A0001FF000C118F101C119F102C11AF103C1F0
:1029B0001BF140D013AADFEF14F0138E139A119C71
:1029C000119A0101800E006F1A0E016F060E026F40
:1029D000000E036F4FC104F150C105F151C106F162
:1029E00052C107F1B3EC1FF003AF05D0AEEC20F0FD
:1029F000118C119A12000E0E3CEC09F0E8CF18F180
:102A00000F0E3CEC09F0E8CF19F1100E3CEC09F088
:102A1000E8CF1AF1110E3CEC09F0E8CF1BF14FC1E1
:102A200000F150C101F151C102F152C103F107821D
:102A3000C0EC1EF018C100F119C101F11AC102F178
:102A40001BC103F112000401730E826F48EC0BF0FE
:102A500004012C0E826F48EC0BF0078462C166F112
:102A600063C167F164C168F165C169F14BC14FF1A0
:102A70004CC150F14DC151F14EC152F157C159F104
:102A800058C15AF1079449EC15F052EC0BF0F5EFF0
:102A900019F066C100F167C101F168C102F169C1B5
:102AA00003F1010151EC20F014EC1EF00401630E5F
:102AB000826F48EC0BF004012C0E826F48EC0BF097
:102AC0004FC100F150C101F151C102F152C103F1F6
:102AD000010151EC20F014EC1EF00401660E826F2F
:102AE00048EC0BF004012C0E826F48EC0BF0AEECBE
:102AF00020F059C100F15AC101F1010151EC20F05F
:102B000014EC1EF00401740E826F48EC0BF01200FE
:102B100010820401530E826F48EC0BF004012C0E5E
:102B2000826F48EC0BF083C32AF184C32BF185C379
:102B30002CF186C32DF187C32EF188C32FF189C3F1
:102B400030F18AC331F18BC332F18CC333F101010F
:102B5000FCEC20F073EC20F000C166F101C167F1DC
:102B600002C168F103C169F18EC32AF18FC32BF151
:102B700090C32CF191C32DF192C32EF193C32FF189
:102B800094C330F195C331F196C332F197C333F159
:102B90000101FCEC20F073EC20F000C14FF101C109
:102BA00050F102C151F103C152F1EFEC20F099C391
:102BB0002FF19AC330F19BC331F19CC332F19DC315
:102BC00033F10101FCEC20F073EC20F000C159F16D
:102BD00001C15AF149EC15F004012C0E826F48EC4A
:102BE0000BF003EF16F0118E19A002D019AE108C65
:102BF00018BE02D018A4108E03018251520A02E1BD
:102C00000F8201D00F928251750A02E1108401D027
:102C100010948251550A02E1108601D0109683511A
:102C2000310A03E11382138402D01392139411A08A
:102C300003D011A401D01084078410B281EF16F0E4
:102C400010A465EF16F0BAC166F1BBC167F1BCC153
:102C500068F1BDC169F1BEC16AF1BFC16BF1C0C10C
:102C60006CF1C1C16DF1C2C16EF1C3C16FF1C4C1DC
:102C700070F1C5C171F1C6C172F1C7C173F1C8C1AC
:102C800074F1C9C175F1CAC176F1CBC177F1CCC17C
:102C900078F1CDC179F1CEC17AF1CFC17BF1D0C14C
:102CA0007CF1D1C17DF1D2C17EF1D3C17FF1D4C11C
:102CB00080F1D5C181F1D6C182F1D7C183F1D8C1EC
:102CC00084F1D9C185F16DEF16F062C166F163C17F
:102CD00067F164C168F165C169F1BAC186F1BBC130
:102CE00087F1BCC188F1BDC189F14BC14FF14CC125
:102CF00050F14DC151F14EC152F157C159F158C176
:102D00005AF107940FA0A3EF16F00101966790EF18
:102D100016F0976790EF16F0986790EF16F09967A6
:102D200094EF16F0A3EF16F027EC14F096C104F11F
:102D300097C105F198C106F199C107F1B3EC1FF0F5
:102D400003BFB9EF19F027EC14F00101000E046F76
:102D5000000E056F010E066F000E076FE4EC1FF00A
:102D600011A02AD011A228D051EC20F0296701D05F
:102D700005D004012D0E826F48EC0BF030C182F4B7
:102D80000401300E822748EC0BF031C182F40401BB
:102D9000300E822748EC0BF032C182F40401300E71
:102DA000822748EC0BF033C182F40401300E8227F5
:102DB00048EC0BF052EC0BF012A8C5D012981AC0D8
:102DC0001BF01B3A1B42070E1B1600011B50000A8A
:102DD000D8B46FEF17F000011B50010AD8B4FBEF15
:102DE00016F000011B50020AD8B4F9EF16F0A1EF5B
:102DF00017F0A1EF17F0AEEC20F02AC001F12BC0C4
:102E000000F1D89001330033D89001330033010131
:102E1000630E046F000E056F000E066F000E076F45
:102E2000E4EC1FF0280E046F000E056F000E066F15
:102E3000000E076FB3EC1FF000C12DF0AEEC20F0D8
:102E400028C001F1019F019D29C000F10101A40EDC
:102E5000046F000E056F000E066F000E076FE4ECA6
:102E60001FF000C12CF000C104F101C105F102C145
:102E700006F103C107F1640E006F000E016F000E32
:102E8000026F000E036FB3EC1FF0050E046F000E0F
:102E9000056F000E066F000E076FE4EC1FF000C117
:102EA00004F101C105F102C106F103C107F1AEEC65
:102EB00020F02DC000F1B3EC1FF000C12EF02EC0A9
:102EC000E8FF050F2D5C03E78A84A1EF17F02EC001
:102ED000E8FF0A0F2D5C01E68A94A1EF17F000C10C
:102EE00024F101C125F102C126F103C127F1AEECA5
:102EF00020F0B4EC20F01A501F0BE8CF00F10101D4
:102F0000640E046F000E056F000E066F000E076F53
:102F1000C4EC1FF024C104F125C105F126C106F15E
:102F200027C107F1B3EC1FF003BF02D08A9401D090
:102F30008A8424C100F125C101F126C102F127C113
:102F400003F1F5EF19F000C124F101C125F102C12F
:102F500026F103C127F110AE4DD0109E00C108F13B
:102F600001C109F102C10AF103C10BF151EC20F0DA
:102F700030C1DAF131C1DBF132C1DCF133C1DDF155
:102F800008C100F109C101F10AC102F10BC103F14D
:102F900001016C0E046F070E056F000E066F000E28
:102FA000076FB3EC1FF003BF04D00101550EDE6FB5
:102FB0001CD008C100F109C101F10AC102F10BC125
:102FC00003F10101A40E046F060E056F000E066FDB
:102FD000000E076FB3EC1FF003BF04D001017F0E9A
:102FE000DE6F03D00101FF0EDE6F1C8E11AEB9EF54
:102FF00019F0119E24C100F125C101F126C102F191
:1030000027C103F111A005D011A203D00FB0B9EF71
:1030100019F010A413EF18F00401750E826F48EC3C
:103020000BF018EF18F00401720E826F48EC0BF0F1
:1030300004012C0E826F48EC0BF051EC20F0296754
:1030400027EF18F00401200E826F2AEF18F0040118
:103050002D0E826F48EC0BF030C182F40401300E6B
:10306000822748EC0BF031C182F40401300E822734
:1030700048EC0BF004012E0E826F48EC0BF032C1CD
:1030800082F40401300E822748EC0BF033C182F445
:103090000401300E822748EC0BF004016D0E826FA4
:1030A00048EC0BF004012C0E826F48EC0BF04FC182
:1030B00000F150C101F151C102F152C103F101010E
:1030C00051EC20F014EC1EF00401480E826F48EC25
:1030D0000BF004017A0E826F48EC0BF004012C0E09
:1030E000826F48EC0BF066C100F167C101F168C165
:1030F00002F169C103F1010151EC20F014EC1EF062
:103100000401630E826F48EC0BF004012C0E826FF9
:1031100048EC0BF066C100F167C101F168C102F132
:1031200069C103F101010A0E046F000E056F000E64
:10313000066F000E076FC4EC1FF0000E046F120E36
:10314000056F000E066F000E076FE4EC1FF051ECE8
:1031500020F02AC182F40401300E822748EC0BF0E3
:103160002BC182F40401300E822748EC0BF02CC1F5
:1031700082F40401300E822748EC0BF02DC182F45A
:103180000401300E822748EC0BF02EC182F40401BA
:10319000300E822748EC0BF02FC182F40401300E70
:1031A000822748EC0BF030C182F40401300E8227F4
:1031B00048EC0BF004012E0E826F48EC0BF031C18D
:1031C00082F40401300E822748EC0BF032C182F405
:1031D0000401300E822748EC0BF033C182F4040165
:1031E000300E822748EC0BF00401730E826F48EC1E
:1031F0000BF004012C0E826F48EC0BF0AEEC20F0CB
:1032000059C100F15AC101F11FEC1BF013A258EF94
:1032100019F004012C0E826F48EC0BF086C166F1A8
:1032200087C167F188C168F189C169F127EC14F0A1
:103230000101000E046F000E056F010E066F000EF7
:10324000076FE4EC1FF051EC20F029672DEF19F027
:103250000401200E826F30EF19F004012D0E826FF1
:1032600048EC0BF030C182F40401300E822748ECA8
:103270000BF031C182F40401300E822748EC0BF0D0
:1032800004012E0E826F48EC0BF032C182F404016F
:10329000300E822748EC0BF033C182F40401300E6B
:1032A000822748EC0BF004016D0E826F48EC0BF0A6
:1032B00013A47FEF19F004012C0E826F48EC0BF081
:1032C00013AC6DEF19F00401500E826F48EC0BF057
:1032D000139C1398139A7FEF19F013AE7AEF19F03D
:1032E0000401460E826F48EC0BF0139E1398139A5C
:1032F0007FEF19F00401530E826F48EC0BF00FB210
:1033000085EF19F00FA0B7EF19F004012C0E826FB2
:1033100048EC0BF0200EF86EF76AF66A040109001B
:10332000F5CF82F448EC0BF00900F5CF82F448ECBD
:103330000BF00900F5CF82F448EC0BF00900F5CF53
:1033400082F448EC0BF00900F5CF82F448EC0BF066
:103350000900F5CF82F448EC0BF00900F5CF82F4B8
:1033600048EC0BF00900F5CF82F448EC0BF052EC7E
:103370000BF00F90109E1298F5EF19F00401630EF8
:10338000826F48EC0BF004012C0E826F48EC0BF0BE
:10339000FBEC19F004012C0E826F48EC0BF06EEC84
:1033A0001AF004012C0E826F48EC0BF0EAEC1AF0D4
:1033B00004012C0E826F48EC0BF00101F80E006F37
:1033C000CD0E016F660E026F030E036F10EC1AF044
:1033D00004012C0E826F48EC0BF000EC1BF052EC59
:1033E0000BF0F5EF19F052EC0BF00301C26B0790F4
:1033F000109204EF1DF0D8900E0E3CEC09F0E8CFCF
:1034000000F10F0E3CEC09F0E8CF01F1100E3CEC9E
:1034100009F0E8CF02F1110E3CEC09F0E8CF03F11E
:103420000101000E046F000E056F010E066F000E05
:10343000076FE4EC1FF051EC20F02AC182F4040184
:10344000300E822748EC0BF02BC182F40401300EC1
:10345000822748EC0BF02CC182F40401300E822745
:1034600048EC0BF02DC182F40401300E822748ECA9
:103470000BF02EC182F40401300E822748EC0BF0D1
:103480002FC182F40401300E822748EC0BF030C1CA
:1034900082F40401300E822748EC0BF031C182F433
:1034A0000401300E822748EC0BF004012E0E826FCF
:1034B00048EC0BF032C182F40401300E822748EC54
:1034C0000BF033C182F40401300E822748EC0BF07C
:1034D00004016D0E826F48EC0BF01200120E3CECF2
:1034E00009F0E8CF00F1130E3CEC09F0E8CF01F150
:1034F000140E3CEC09F0E8CF02F1150E3CEC09F09B
:10350000E8CF03F101010A0E046F000E056F000EF3
:10351000066F000E076FC4EC1FF0000E046F120E52
:10352000056F000E066F000E076FE4EC1FF051EC04
:1035300020F02AC182F40401300E822748EC0BF0FF
:103540002BC182F40401300E822748EC0BF02CC111
:1035500082F40401300E822748EC0BF02DC182F476
:103560000401300E822748EC0BF02EC182F40401D6
:10357000300E822748EC0BF02FC182F40401300E8C
:10358000822748EC0BF030C182F40401300E822710
:1035900048EC0BF004012E0E826F48EC0BF031C1A9
:1035A00082F40401300E822748EC0BF032C182F421
:1035B0000401300E822748EC0BF033C182F4040181
:1035C000300E822748EC0BF00401730E826F48EC3A
:1035D0000BF012000A0E3CEC09F0E8CF00F10B0EE4
:1035E0003CEC09F0E8CF01F10C0E3CEC09F0E8CF1F
:1035F00002F10D0E3CEC09F0E8CF03F11FEF1BF0D8
:10360000060E3CEC09F0E8CF00F1070E3CEC09F0A7
:10361000E8CF01F1080E3CEC09F0E8CF02F1090E09
:103620003CEC09F0E8CF03F11FEF1BF00101AEEC19
:1036300020F0078457C100F158C101F1079401013E
:10364000E80E046F800E056F000E066F000E076F08
:10365000C4EC1FF0000E046F040E056F000E066F21
:10366000000E076FE4EC1FF0880E046F130E056F59
:10367000000E066F000E076FB3EC1FF00A0E046F0A
:10368000000E056F000E066F000E076FE4EC1FF0D2
:1036900051EC20F00101296753EF1BF00401200ECB
:1036A000826F56EF1BF004012D0E826F48EC0BF079
:1036B00030C182F40401300E822748EC0BF031C196
:1036C00082F40401300E822748EC0BF032C182F400
:1036D0000401300E822748EC0BF004012E0E826F9D
:1036E00048EC0BF033C182F40401300E822748EC21
:1036F0000BF00401430E826F48EC0BF0120087C3FD
:103700002AF188C32BF189C32CF18AC32DF18BC315
:103710002EF18CC32FF18DC330F18EC331F190C3E4
:1037200032F191C333F10101296BFCEC20F073EC11
:1037300020F00101000E046F000E056F010E066FF0
:10374000000E076FC4EC1FF00E0E0C6E00C10BF0E4
:1037500025EC09F00F0E0C6E01C10BF025EC09F001
:10376000100E0C6E02C10BF025EC09F0110E0C6E60
:1037700003C10BF025EC09F004017A0E826F48ECCE
:103780000BF004012C0E826F48EC0BF00401350E97
:10379000826F48EC0BF004012C0E826F48EC0BF0AA
:1037A000FBEC19F0FDEF13F087C32AF188C32BF16E
:1037B00089C32CF18AC32DF18BC32EF18CC32FF159
:1037C0008DC330F18EC331F190C332F191C333F127
:1037D0000101296BFCEC20F073EC20F0880E046FE3
:1037E000130E056F000E066F000E076FB8EC1FF08A
:1037F000000E046F040E056F000E066F000E076FBB
:10380000C4EC1FF00101E80E046F800E056F000E7E
:10381000066F000E076FE4EC1FF00A0E0C6E00C17D
:103820000BF025EC09F00B0E0C6E01C10BF025EC32
:1038300009F00C0E0C6E02C10BF025EC09F00D0E18
:103840000C6E03C10BF025EC09F004017A0E826FB7
:1038500048EC0BF004012C0E826F48EC0BF00401D5
:10386000360E826F48EC0BF004012C0E826F48EC90
:103870000BF0EAEC1AF0FDEF13F087C32AF188C3CE
:103880002BF189C32CF18AC32DF18BC32EF18CC38C
:103890002FF18DC330F18FC331F190C332F191C359
:1038A00033F10101FCEC20F073EC20F0000E046F0A
:1038B000120E056F000E066F000E076FC4EC1FF0AE
:1038C00001010A0E046F000E056F000E066F000E58
:1038D000076FE4EC1FF0120E0C6E00C10BF025EC2C
:1038E00009F0130E0C6E01C10BF025EC09F0140E5B
:1038F0000C6E02C10BF025EC09F0150E0C6E03C125
:103900000BF025EC09F004017A0E826F48EC0BF005
:1039100004012C0E826F48EC0BF00401370E826F0D
:1039200048EC0BF004012C0E826F48EC0BF06EECAF
:103930001AF0FDEF13F087C32AF188C32BF189C376
:103940002CF18AC32DF18BC32EF18CC32FF18DC3C3
:1039500030F18EC331F190C332F191C333F10101E3
:10396000296BFCEC20F073EC20F0880E046F130E32
:10397000056F000E066F000E076FB8EC1FF0000E0B
:10398000046F040E056F000E066F000E076FC4EC87
:103990001FF00101E80E046F800E056F000E066F28
:1039A000000E076FE4EC1FF0060E0C6E00C10BF06A
:1039B00025EC09F0070E0C6E01C10BF025EC09F0A7
:1039C000080E0C6E02C10BF025EC09F0090E0C6E0E
:1039D00003C10BF025EC09F004017A0E826F48EC6C
:1039E0000BF004012C0E826F48EC0BF00401380E32
:1039F000826F48EC0BF004012C0E826F48EC0BF048
:103A000000EC1BF0FDEF13F081B803D02FB0C2EF34
:103A10001DF007A87CEF1DF00101800E006F1A0E4B
:103A2000016F060E026F000E036F4BC104F14CC113
:103A300005F14DC106F14EC107F1B3EC1FF003BF14
:103A4000C2EF1DF00EEC1EF04BC100F14CC101F1B4
:103A50004DC102F14EC103F10782C0EC1EF018C146
:103A600004F119C105F11AC106F11BC107F1F80EE5
:103A7000006FCD0E016F660E026F030E036FB3EC85
:103A80001FF00E0E0C6E00C10BF025EC09F00F0EAE
:103A90000C6E01C10BF025EC09F0100E0C6E02C18A
:103AA0000BF025EC09F0110E0C6E03C10BF025ECA8
:103AB00009F007840101AEEC20F057C100F158C1B4
:103AC00001F107940A0E0C6E00C10BF025EC09F011
:103AD0000B0E0C6E01C10BF025EC09F00C0E0C6EF8
:103AE00002C10BF025EC09F00D0E0C6E03C10BF0BA
:103AF00025EC09F0C2EF1DF007AAC2EF1DF0078404
:103B00000101AEEC20F057C100F158C101F107945A
:103B1000060E0C6E00C10BF025EC09F0070E0C6EC2
:103B200001C10BF025EC09F0080E0C6E02C10BF080
:103B300025EC09F0090E0C6E03C10BF025EC09F021
:103B4000078462C100F163C101F164C102F165C182
:103B500003F10794120E0C6E00C10BF025EC09F076
:103B6000130E0C6E01C10BF025EC09F0140E0C6E57
:103B700002C10BF025EC09F0150E0C6E03C10BF021
:103B800025EC09F00798079A0401805181197F0BF1
:103B90000DE09EA8FED714EE00F081517F0BE126C8
:103BA000E750812B0F01AD6EC4EF1DF09FEF0AF0BF
:103BB00018C100F119C101F11AC102F11BC103F1D1
:103BC000000E046F000E056F010E066F000E076FEA
:103BD000E4EC1FF029A103EF1EF02051D8B403EF4D
:103BE0001EF018C100F119C101F11AC102F11BC187
:103BF00003F1000E046F000E056F0A0E066F000E33
:103C0000076FE4EC1FF0120001010451001305518D
:103C10000113065102130751031312000101186B1F
:103C2000196B1A6B1B6B12002AC182F40401300E4F
:103C3000822748EC0BF02BC182F40401300E82275E
:103C400048EC0BF02CC182F40401300E822748ECC2
:103C50000BF02DC182F40401300E822748EC0BF0EA
:103C60002EC182F40401300E822748EC0BF02FC1E4
:103C700082F40401300E822748EC0BF030C182F44C
:103C80000401300E822748EC0BF031C182F40401AC
:103C9000300E822748EC0BF032C182F40401300E62
:103CA000822748EC0BF033C182F40401300E8227E6
:103CB00048EC0BF012002FC182F40401300E822771
:103CC00048EC0BF030C182F40401300E822748EC3E
:103CD0000BF031C182F40401300E822748EC0BF066
:103CE00032C182F40401300E822748EC0BF033C15C
:103CF00082F40401300E822748EC0BF01200060E0D
:103D00001E6E060E1F6E060E206E1E2E85EF1EF016
:103D10001F2E85EF1EF0202E85EF1EF08B84020EE5
:103D20001E6E020E1F6E020E206E1E2E95EF1EF0EE
:103D30001F2E95EF1EF0202E95EF1EF08B94120093
:103D4000FF0E1F6E1FC020F0030E1E6E8B841E2EF2
:103D5000A6EF1EF0030E1E6E202EA6EF1EF08B9413
:103D60001FC020F0030E1E6E1E2EB4EF1EF0030EB9
:103D70001E6E203EB4EF1EF01F2EA2EF1EF01200AA
:103D80000101005305E1015303E1025301E1002B5E
:103D900083EC1FF0AEEC20F03951006F3A51016F07
:103DA000420E046F4B0E056F000E066F000E076F7C
:103DB000C4EC1FF000C104F101C105F102C106F11C
:103DC00003C107F118C100F119C101F11AC102F1D3
:103DD0001BC103F107B2F1EF1EF0B8EC1FF0F3EFD7
:103DE0001EF0B3EC1FF000C118F101C119F102C1BE
:103DF0001AF103C11BF11200AEEC20F059C100F121
:103E00005AC101F1060E3CEC09F0E8CF04F1070EAF
:103E10003CEC09F0E8CF05F1080E3CEC09F0E8CFE6
:103E200006F1090E3CEC09F0E8CF07F1B3EC1FF006
:103E300000C124F101C125F102C126F103C127F11E
:103E4000290E046F000E056F000E066F000E076F3F
:103E5000C4EC1FF0EE0E046F430E056F000E066FEC
:103E6000000E076FB8EC1FF024C104F125C105F165
:103E700026C106F127C107F1C4EC1FF000C11CF1F7
:103E800001C11DF102C11EF103C11FF1120E3CEC74
:103E900009F0E8CF04F1130E3CEC09F0E8CF05F18E
:103EA000140E3CEC09F0E8CF06F1150E3CEC09F0DD
:103EB000E8CF07F10D0E006F000E016F000E026FCC
:103EC000000E036FC4EC1FF0180E046F000E056F98
:103ED000000E066F000E076FE4EC1FF01CC104F12A
:103EE0001DC105F11EC106F11FC107F1B8EC1FF09D
:103EF0006A0E046F2A0E056F000E066F000E076F24
:103F0000B3EC1FF01200BF0EFA6E200E3A6F396B41
:103F1000D8900037013702370337D8B094EF1FF03D
:103F20003A2F89EF1FF039073A070353D8B412002C
:103F30000331070B80093F6F03390F0B010F396FF6
:103F400080EC5FF0406F390580EC5FF0405D405FD2
:103F5000396B3F33D8B0392739333FA9A9EF1FF068
:103F60004051392712000101D3EC20F0D8B01200E3
:103F7000010103510719346F96EC20F0D8900751D6
:103F8000031934AF800F12000101346BBAEC20F03A
:103F9000D8A0D0EC20F0D8B01200A5EC20F0AEEC08
:103FA00020F01F0E366FE6EC20F00B35D8B096EC03
:103FB00020F0D8A00335D8B01200362FD3EF1FF071
:103FC00034B1BDEC20F012000101346B0451051135
:103FD000061107110008D8A0BAEC20F0D8A0D0EC48
:103FE00020F0D8B01200086B096B0A6B0B6BE6EC83
:103FF00020F01F0E366FE6EC20F007510B5DD8A4C1
:104000000EEF20F006510A5DD8A40EEF20F0055106
:10401000095DD8A40EEF20F00451085DD8A021EF6F
:1040200020F00451085F0551D8A0053D095F0651F5
:10403000D8A0063D0A5F0751D8A0073D0B5FD89076
:104040000081362FFBEF1FF034B1BDEC20F0346B54
:10405000BAEC20F0D890EAEC20F007510B5DD8A420
:104060003EEF20F006510A5DD8A43EEF20F0055146
:10407000095DD8A43EEF20F00451085DD8A04DEFB3
:1040800020F0003F4DEF20F0013F4DEF20F0023FC8
:104090004DEF20F0032BD8B4120034B1BDEC20F06A
:1040A00012000101346BBAEC20F0D8B01200EFEC32
:1040B00020F0200E366F003701370237033711EE3C
:1040C00033F00A0E376FE7360A0EE75CD8B0E76EBA
:1040D000E552372F63EF20F0362F5BEF20F034B13D
:1040E0002981D890120001010A0E346F200E366F1C
:1040F00011EE29F03451376F0A0ED890E652D8B03D
:10410000E726E732372F7EEF20F003330233013307
:104110000033362F78EF20F0E750FF0FD8A003359B
:10412000D8B0120029B1BDEC20F0120004510027D4
:104130000551D8B0053D01270651D8B0063D0227EC
:104140000751D8B0073D032712000051086F0151F5
:10415000096F02510A6F03510B6F12000101006BCE
:10416000016B026B036B12000101046B056B066BA4
:10417000076B12000335D8A012000351800B001FFB
:10418000011F021F031F003FCDEF20F0013FCDEFC5
:1041900020F0023FCDEF20F0032B342B032512003B
:1041A0000735D8A012000751800B041F051F061FFA
:1041B000071F043FE3EF20F0053FE3EF20F0063F49
:1041C000E3EF20F0072B342B0725120000370137CF
:1041D00002370337083709370A370B371200010156
:1041E000296B2A6B2B6B2C6B2D6B2E6B2F6B306B13
:1041F000316B326B336B120001012A510F0B2A6FA6
:104200002B510F0B2B6F2C510F0B2C6F2D510F0BB4
:104210002D6F2E510F0B2E6F2F510F0B2F6F305113
:104220000F0B306F31510F0B316F32510F0B326F5B
:1042300033510F0B336F120000011650FF0A01E1DA
:104240001200390EC86E800EC76E280EC66E000EA4
:10425000C56E1550000AD8B457EF21F01550010A69
:10426000D8B470EF21F01550020AD8B489EF21F0CC
:104270001550030AD8B4A2EF21F01550040AD8B49F
:10428000CAEF21F01550050AD8B4E3EF21F015501C
:10429000060AD8B4FCEF21F01550070AD8B415EF80
:1042A00022F01550080AD8B42EEF22F01200165052
:1042B000000AD8B44DEF22F01650010AD8B451EFDD
:1042C00022F01650020AD8B455EF22F01650030A15
:1042D000D8B459EF22F01650040AD8B4CCEF22F02B
:1042E0001650000AD8B461EF22F01650010AD8B473
:1042F00065EF22F01650020AD8B469EF22F016508A
:10430000030AD8B46DEF22F01650040AD8B4CCEFEB
:1043100022F01650000AD8B471EF22F01650010AAC
:10432000D8B475EF22F01650020AD8B479EF22F013
:104330001650030AD8B47DEF22F01650040AD8B400
:10434000CCEF22F01650000AD8B48AEF22F01650B3
:10435000010AD8B48EEF22F01650020AD8B492EFB8
:1043600022F01650030AD8B4A6EF22F01650040A21
:10437000D8B4AAEF22F01650050AD8B4AEEF22F056
:104380001650060AD8B4B2EF22F01650070AD8B475
:10439000B5EF22F01650000AD8B4B9EF22F016504B
:1043A000010AD8B4BDEF22F01650020AD8B4C1EF0A
:1043B00022F01650030AD8B4C5EF22F01650040AB2
:1043C000D8B4C8EF22F01650000AD8B4D0EF22F0CB
:1043D0001650010AD8B4D4EF22F01650020AD8B40D
:1043E000D8EF22F01650030AD8B4DCEF22F01650B2
:1043F000040AD8B4CCEF22F01650000AD8B4E6EF85
:1044000022F01650010AD8B4EAEF22F01650020A40
:10441000D8B4EEEF22F01650030AD8B4F2EF22F02F
:104420001650040AD8B4CCEF22F01650000AD8B4C3
:10443000F3EF22F01650010AD8B4F7EF22F016502D
:10444000020AD8B4FBEF22F01650030AD8B4FFEFEB
:1044500022F01650040AD8B4CCEF22F01650000A0D
:10446000D8B400EF23F01650010AD8B404EF23F0BB
:104470001650020AD8B408EF23F01650030AD8B435
:104480000CEF23F01650040AD8B40DEF23F01650A9
:10449000050AD8B410EF23F012009E96C580162AA4
:1044A0001200E20EC96E162A1200770EC96E162A85
:1044B0001200020EE86E8AB4E88AE8CFC9FF162A15
:1044C00012009E96C580162A1200E20EC96E162AA8
:1044D0001200790EC96E162A1200000EC96E162A35
:1044E00012009E96C580162A1200E20EC96E162A88
:1044F00012007A0EC96E162A120018BC03D0DEC153
:10450000E8FF04D01850E844E8441F09E8CFC9FF89
:10451000162A12009E96C580162A1200E20EC96E57
:10452000162A120011BA03D011BC01D003D0050E17
:10453000156E3ED00101DA67A2EF22F0100EC96EAF
:10454000A4EF22F0DAC1C9FF162A1200DBC1C9FFAD
:10455000162A1200DCC1C9FF162A1200DDC1C9FFEC
:10456000162A1200C584162A1200FF0E166E1D9E12
:1045700012009E96C580162A1200E20EC96E162AF7
:104580001200760EC96E162A1200C584162A120071
:10459000FF0E166E1D9E1200C584152A166A1200A3
:1045A0009E96C580162A1200E20EC96E162A1200C7
:1045B0007B0EC96E162A120011AA04D0230EC96EF2
:1045C000162A12001C0EC96E162A12009E96C5806D
:1045D000162A1200E20EC96E162A12007C0EC96E4F
:1045E000162A1200E9D79E96C580162A1200E20EFE
:1045F000C96E162A12007D0EC96E162A1200DCD76B
:104600009E96C580162A1200E20EC96E162A120066
:104610007E0EC96E162A1200CFD7C584162A120044
:10462000FF0E166E1D9E12001650FF0AD8B4D2EF70
:1046300023F0390EC86E800EC76E280EC66E000EAF
:10464000C56E1550000AD8B42DEF23F01550010A9D
:10465000D8B441EF23F0D2EF23F01650000AD8B4BB
:104660007FEF23F01650010AD8B483EF23F01650E1
:10467000020AD8B48DEF23F01650030AD8B490EF95
:1046800023F01650000AD8B496EF23F01650010A12
:10469000D8B49AEF23F01650020AD8B4A4EF23F04E
:1046A0001650030AD8B4A7EF23F01650040AD8B462
:1046B000ADEF23F01650050AD8B4B0EF23F0165032
:1046C000060AD8B4B6EF23F01650070AD8B4B9EFEB
:1046D00023F01650080AD8B4BFEF23F01650090A89
:1046E000D8B4C2EF23F016500A0AD8B4C8EF23F0AA
:1046F00016500B0AD8B4CBEF23F0D2EF23F09E96DE
:10470000C580D1EF23F017B004D04E0EC96ED1EFA3
:1047100023F0500EC96ED1EF23F0C584D1EF23F002
:10472000152AFF0E166E1280D2EF23F09E96C580DA
:10473000D1EF23F017B004D04F0EC96ED1EF23F0A4
:10474000510EC96ED1EF23F0C586D1EF23F0C9CF4A
:1047500024F0C59AC588D1EF23F0C586D1EF23F0A8
:10476000C9CF25F0C59AC588D1EF23F0C586D1EF12
:1047700023F0C9CF26F0C59AC588D1EF23F0C586AE
:10478000D1EF23F0C9CF27F0C58AC588D1EF23F038
:10479000C584D1EF23F0FF0E166E12861D9CD2EF5A
:1047A00023F0162A120012B012D012B213D012B493
:1047B00014D012A6120007B01200129624C028F0DE
:1047C00025C029F026C02AF027C02BF01200129035
:1047D0001282120012921284120000011650FF0A77
:0C47E00004E11294166A14EC23F012009D
:10BF0000E844F926000C160C2B0C3F0C520C640C68
:10BF1000760C860C960CA50CB30CC10CCF0CDC0C6B
:06BF2000E80CF40C000C1B
:00000001FF
